:020000021000EC
:10F8000011241FBECFEFD0E4DEBFCDBF11E0A0E0DA
:10F81000B1E0E4ECFDEF01E00BBF02C007900D92F8
:10F82000A030B107D9F712E0A0E0B1E001C01D920D
:10F83000A030B107E1F70E9454FC0C94E0FE0C9458
:10F8400021FC08958091C80085FFFCCF81E480935E
:10F85000CE008091C80085FFFCCF86E58093CE0066
:10F860008091C80085FFFCCF82E58093CE00809117
:10F87000C80085FFFCCF82E48093CE008091C80051
:10F8800085FFFCCF8FE48093CE008091C80085FF78
:10F89000FCCF8FE48093CE008091C80085FFFCCF21
:10F8A00084E58093CE0008952F923F924F925F920D
:10F8B0006F927F928F929F92AF92BF92CF92DF9280
:10F8C000EF92FF920F931F93DF93CF9300D00F928D
:10F8D000CDB7DEB78FEF87B998B188B984B995B144
:10F8E00085B98AB99BB18BB9299AF894A89584B740
:10F8F000877F84BF80916000886180936000109250
:10F9000060000C98149A1092CD008AE08093CC008D
:10F9100088E18093C90086E08093CA00049B04C0FC
:10F920001498E0E0F0E009952E9820E030E040E502
:10F9300053EC8091C80087FF0AC08091CE008335C8
:10F9400031F40E9422FCAA24BB2419820CC067E077
:10F95000203D360710F0149829982F5F3F4FCA01B9
:10F960000197F1F7E6CF8091C80087FFFCCF2E9A70
:10F970009091CE00913641F48091C80085FFFCCF74
:10F9800089E58093CE00EFCF9134C9F48091C8000F
:10F9900087FFFCCF2E9A2091CE008091C80087FF70
:10F9A000FCCF2E9A9091CE008091C80085FFFCCFAD
:10F9B000322E2224A92EBB24A228B328AEC192360F
:10F9C00099F48091C80085FFFCCFE9E5E093CE0073
:10F9D0008091C80085FFFCCFF1E0F093CE008091CC
:10F9E000C80085FFFCCF75C1923409F0A0C080919A
:10F9F000C80087FFFCCF2E9A9091CE008091C8005E
:10FA000087FFFCCF2E9A8091CE00792E6624282F76
:10FA100030E0262937293B832A838091C80087FF5D
:10FA2000FCCF2E9A9091CE0020E030E0E0E0F1E0B3
:10FA30004A815B812417350710F08FEF07C0809152
:10FA4000C80087FFFCCF2E9A8091CE0080832F5F65
:10FA50003F4F51E02030350711F03196E9CF6981F1
:10FA6000663409F05FC0963409F03CC0750100E0CF
:10FA700010E0EE0CFF1C001F111FA8019701A0E071
:10FA8000B1E08C9190E011965C9011974424842908
:10FA90009529129661E00C01F90140935B00609397
:10FAA0005700E89511242E5F3F4F4F4F5F4F8A81DB
:10FAB0009B8102979B838A83892B19F795E0F70135
:10FAC00000935B0090935700E89507B600FCFDCFCC
:10FAD000E1E1E0935700E8955695479537952795CE
:10FAE00059011BC09534C9F4EA80FB80850120E0F0
:10FAF000C22E21E0D22EF60161916F01C8010E9451
:10FB0000D2FE0F5F1F4F0894E108F108E114F104E1
:10FB100091F72A813B81A20EB31E8091C80085FF18
:10FB2000FCCFBEC08091C80085FFFCCFD2C0973605
:10FB300009F06AC08091C80087FFFCCF2E9A90918F
:10FB4000CE008091C80087FFFCCF2E9A8091CE0016
:10FB5000992E8824C82EDD24C828D9288091C80071
:10FB600087FFFCCF2E9A8091CE00863499F59501BF
:10FB700040E050E0220F331F441F551F2F3F67EF17
:10FB8000360761E0460760E0560718F06FEF7FEF39
:10FB900004C04BBFF901679176918091C80085FF41
:10FBA000FCCF6093CE008091C80085FFFCCF70939E
:10FBB000CE002E5F3F4F4F4F5F4F8EEF9FEFC80E2F
:10FBC000D91EC114D104D1F656954795379527957E
:10FBD0005901C9CE853409F0C6CE76018501C80128
:10FBE0000E94CAFE982F8091C80085FFFCCF909399
:10FBF000CE000F5F1F4F0894E108F108E114F104F3
:10FC000071F7AC0CBD1CAFCE953639F599819634A1
:10FC1000F1F480E090E0A0E0B0E023E0FC01A093EC
:10FC20005B0020935700E89507B600FCFDCF80509D
:10FC30009F4FAF4FBF4F803038EF930731E0A3079E
:10FC400030E0B30751F741E140935700E8958091C8
:10FC5000C80085FFFCCF5DE09AC0953489F488E147
:10FC600090E0ECE00FB6F894A895809360000FBE8A
:10FC7000E09360008091C80085FFFCCFFDE064C088
:10FC8000903541F48091C80085FFFCCF2DE0209392
:10FC9000CE0069CE9C3441F48091C80085FFFCCF32
:10FCA0003DE03093CE005FCE903731F48091C800B4
:10FCB00085FFFCCF43E560C0943771F48091C800A4
:10FCC00085FFFCCF56E45093CE008091C80085FF9D
:10FCD000FCCF1092CE0047CE892F8857823078F41F
:10FCE0008091C80087FFFCCF2E9A8091CE00809132
:10FCF000C80085FFFCCF6DE06093CE0034CE943514
:10FD000081F48091C80087FFFCCF2E9A8091CE00AD
:10FD100089838091C80085FFFCCF9DE09093CE0041
:10FD200022CE933519F40E9422FC1DCE963579F42B
:10FD30008091C80085FFFCCFE0E3E093CE00809186
:10FD4000C80085FFFCCFF8E3F093CE000CCE9337CC
:10FD5000B1F48091C80085FFFCCF25E02093CE0050
:10FD60008091C80085FFFCCF37E93093CE008091A9
:10FD7000C80085FFFCCF4EE14093CE00F4CD9B310F
:10FD800009F4F1CD8091C80085FFFCCF5FE350936B
:10FD9000CE00E9CDF999FECF92BD81BDF89A9927A1
:10FDA00080B50895262FF999FECF1FBA92BD81BD67
:10FDB00020BD0FB6F894FA9AF99A0FBE01960895ED
:04FDC000F894FFCFE5
:040000031000F800F1
:00000001FF
